:020000040800F2
:1000000000200020B12F0008692200086B220008A0
:1000100000000000000000000000000000000000E0
:100020000000000000000000000000006D22000839
:1000300000000000000000006F2200088D4300084F
:10004000213000082130000821300008213000084C
:10005000213000082130000821300008213000083C
:10006000213000082130000821300008213000082C
:10007000A9430008213000082130000811140008AD
:100080002130000821300008000000002130000865
:100090002130000821300008213000082912000812
:1000A00021300008213000082130000821300008EC
:1000B0004543000800000000213000080000000057
:0400C0005FF808F1EC
:1000C40002B4714649084900095C49008E4402BCE7
:1000D4007047C046002243088B4274D303098B4205
:1000E4005FD3030A8B4244D3030B8B4228D3030C04
:1000F4008B420DD3FF22090212BA030C8B4202D3A6
:100104001212090265D0030B8B4219D300E0090ACD
:10011400C30B8B4201D3CB03C01A5241830B8B42D6
:1001240001D38B03C01A5241430B8B4201D34B03BF
:10013400C01A5241030B8B4201D30B03C01A524124
:10014400C30A8B4201D3CB02C01A5241830A8B42A9
:1001540001D38B02C01A5241430A8B4201D34B0292
:10016400C01A5241030A8B4201D30B02C01A5241F6
:10017400CDD2C3098B4201D3CB01C01A52418309AA
:100184008B4201D38B01C01A524143098B4201D3E4
:100194004B01C01A524103098B4201D30B01C01A0F
:1001A4005241C3088B4201D3CB00C01A5241830889
:1001B4008B4201D38B00C01A524143088B4201D3B6
:1001C4004B00C01A5241411A00D201465241104616
:1001D4007047FFE701B5002000F006F802BDC046F5
:1001E4000029F7D076E770477047C0460020704773
:1001F4007047002070477047002070470023024A70
:1002040043708261837070472000002043788B42E2
:1002140005D00022024B1A810123017083707047BC
:10022400DC0200208378002B01D1023383707047F5
:100234008378002B01D10333837070470F21124B55
:1002440070B55D890600ADB22940043000F080FC31
:100254000E4CED06230038331B78ED0F9D420ED073
:10026400002B01D10A4B00E00A4BE069236002F045
:10027400F7F82100E069383402F00CF92570B06910
:100284000368DB68984770BDDC0200205C03002033
:10029400220C94102309720070B5074C8069260063
:1002A4000368543635889B6898473388ADB29D42BD
:1002B40001D15034208070BDDC020020F8B5040068
:1002C4008078C0B204286DD8FFF7FAFE031E474EAB
:1002D40052002000FFF7E0FF334D20002B00503385
:1002E40019880C3009B200F03FFC63892269523549
:1002F400D31A62681BB29B18227A6360134163812C
:100304009B049B0C2B804DE0A06903685B689847B5
:100314002378254D0A2B1AD8244A99008E58002E8A
:1003240015D03371336830001B689847071E0CD111
:100334002000A661FFF782FFA06903681B69984744
:10034400A88158352F8004232BE0194BA361543521
:100354002B8801339BB22B8022E0A06903681B69C0
:100364009847114B98811BE02000FFF767FF17E0C7
:100374002000FFF791FF0C4B1A0058321288002A14
:1003840010D02278627092B21A81012250331B88F5
:100394002275227A1BB2A381236163819340636037
:1003A4000023A370F8BDC046DC020020143200080C
:1003B40020000020034A044B1A60044A044B1A60CC
:1003C4007047C046003200082000002028000020AA
:1003D400440000202021044A138801331380034A77
:1003E40013880B4313807047480000204A00002004
:1003F4000300FF339B790079181A80B2704702001A
:100404000379FF3291795A1C0271994202D9C018BA
:10041400807900E000207047020010B5FF32937924
:10042400FF2B03D05C1CC3189471997110BD02009A
:10043400FF329279030082180020934204D0997904
:1004440001334018C0B2F8E77047000010B50C2320
:1004540000220349034801F051FD00F037FA10BDB2
:10046400583200084C00002000B50A4BC3B06A465D
:10047400009343235371002313710122FF336B4410
:100484009A716B469871044B6946186800F0ECF950
:1004940043B000BD4832000898020020024B034AD2
:1004A4001A60034A5A6070474C0000201443000845
:1004B40000440040052010B5404202F059FA0548B6
:1004C40002F064FA012002F07BFA012002F064FADF
:1004D40010BDC046808D5B00012330B5084C094A2D
:1004E40023602368084953438D685B1B06256843D2
:1004F400181823688D6853435B1B9842F9D830BDA4
:1005040078020020808D5B0010E000E0012330B50C
:10051400084C094A23602368084953438D685B1BD0
:10052400074D6843181823688D6853435B1B984232
:10053400F9D830BD78020020808D5B0010E000E027
:1005440070170000704770477047704770477047D6
:100554000B4A0C4B5089191DC8871089991DC887EF
:100564001900D0880831C88719009088483108805C
:10057400190050884A31088012884C331A80704719
:10058400ACF7FF1FDC02002010B50B4802F0F8FBAB
:1005940002F032F80020094B18605860986002F0AD
:1005A4005BF8012383F31088054B1B6883F30888E9
:1005B400044B1B68984710BD0038014010E000E070
:1005C40000ECFF1F04ECFF1F10B5012802D101F05D
:1005D400EBFCFEE7FFF7D8FF10BD00207047704723
:1005E400F0B5060080208BB00121800202F00EF9E4
:1005F40080200121800002F015F9902003230025BA
:10060400012702A9C0050B7104ACCD71029701F05A
:10061400B5FE1C4801F03EFE200001F063FE2100FF
:10062400184804952771A5602561656101F044FEB1
:1006340039000722134801F065FE124801F067FEF5
:100644003900104801F056FE01210E4801F086FEE3
:100654000028F9D00C23012401A80370093B43703E
:10066400847001F09DFF220000240421054801F05C
:100674006CFEB460B481034801F05FFE20000BB04F
:10068400F0BDC0460024014007B50021094801F02F
:1006940031FE684601F0AEFE902001236946C00594
:1006A400009301F06BFE0449024801F057FE012853
:1006B400F9D007BD002401400100000170B5818913
:1006C4000400104E002914D080250F4B6D01DD6706
:1006D40083689800FFF7FEFC330058331A8880B211
:1006E400013292B21A800023A360A381074B1D60DC
:1006F40006E03300080054331A88013292B21A809B
:1007040070BDC046DC02002004E100E000E100E02E
:10071400024B034A083313607047C04698320008FE
:1007240084020020036870B505005B6898472B6855
:1007340004005B68280098470002041920B270BDC9
:1007440070B505000C000368C9B29B6898472B6814
:1007540024122800E1B29B68984770BDF8B50400E4
:1007640000680E000368DB689847002872D025797A
:10077400012D16D0002D02D0022D33D06AE020685E
:1007840003685B689847030020683E2B05D1036823
:100794001B689847012323715AE003685B699847F3
:1007A40056E020680368DB689847022852D920681D
:1007B40003681B6898472072206803681B68984781
:1007C40080B2E080257A2068E388ED180368EDB2F2
:1007D4001B68984785423FD1E388FF2B3CD802230E
:1007E400237137E02068E5880368ADB2DB68984779
:1007F40085422FDA237A350073710023FF35AB71FC
:100804003371E288A9793368914208D220689F68DD
:1008140003681B68984701003000B847F1E70025DA
:10082400DB683000257198470600206803681B6860
:10083400984786420AD120210A4A206813888B43AC
:10084400138003689B699847012009E0FFF7C2FD04
:10085400280005E0002003E0FFF7BCFD0020207124
:10086400F8BDC0464A000020F8B50D002F0004680A
:100874003E21236820009B689847236869799B6818
:10088400200098472368FF37B9799B682000984770
:10089400BB7969792000C9182368C9B29B68984755
:1008A4000026BA792368B24207D9AA1991799B68BC
:1008B400200001369847F6B2F3E79E682B682800BB
:1008C400DB68984701002000B047F8BD044B054A97
:1008D40005491A6000221A710A70044A13607047AD
:1008E400A00200204C0000209C020020980200205E
:1008F40030B50400407987B042380023142800D969
:10090400DAE0FFF7DDFB9C7ED94BD977D9D9D9D969
:10091400D9B3C9D932D9D9D9D98B0B002200FF3226
:1009240093712371236855219B68200098478D217A
:100934002000FFF705FF236800219B6820009847EB
:10094400AA212000FFF7FCFE2368FF219B682000FA
:1009540098470C25013DEDB2002D00D19AE02368A3
:1009640000219B6820009847F4E72000FFF7DAFE97
:1009740005002000FFF7D6FE2300FF3322799B7980
:1009840000249A4200D098E04D4B81B2AAB2186874
:1009940000F0B6FD5020FFF767FD8EE023682000CD
:1009A4005B689847464B041E1B68039310D00124D0
:1009B40018001C70002100F0EDFD2100414802F0F8
:1009C400E3F8902022000421C00501F031FD0FE07E
:1009D400020090200421C00501F02AFD21000398A3
:1009E40000F0D8FD039B21001C70364802F0CCF8BF
:1009F400452010E02200FF3293712371324B5233B1
:100A040043E0236820005B689847304B81B2186844
:100A1400FFF7FCFB4320FFF727FD4DE022000025F4
:100A2400FF32937123712B00274A4233D15C236830
:100A340020009B6801359847062DF4D12AE00E2545
:100A4400236820005B68984702ABED18022302007C
:100A5400009331212B001E4800F03CF922000023B2
:100A6400FF32937123710023E95E10E023682000B4
:100A74005B68984723000022FF339A712271154B5B
:100A84003F2802D8104A40008318198809B2200070
:100A9400FFF756FE012410E022000025FF32937177
:100AA4002371094B2000EB181988023509B2FFF7AE
:100AB40047FE802DF5D1EDE70024200007B030BDBE
:100AC400A8030020002C0140DC0200204400002088
:100AD400CC0200201C00002030B5174BC3B000939B
:100AE4000023164C23702178154D164800291AD17D
:100AF40003682860002B13D00322134802F034FB50
:100B040069462868FFF72AFE002809D06846FFF7DF
:100B1400EFFE0028F4D069462868FFF7A5FEEFE74A
:100B240023780133DEE70C22084B1B785343C318A8
:100B34002B6043B030BDC046483200089402002008
:100B440098020020A0020020AC0200209C02002099
:100B5400037902688B4202D2CB1A9A4001E05B1AF5
:100B64001A41026001717047037A002B15D0038883
:100B74000180CB1A80219BB21AB289018A4201DD1D
:100B8400084A04E008498A4203DA8022D2019B1809
:100B94001AB243689B18436003E00123018041605B
:100BA4000372704700C0FFFF00E0FFFFF7B50500C8
:100BB40080200121C00201F029FE6A46022313713C
:100BC400013353718023002401261B4FDB003800BE
:100BD40069469671D471009301F0D0FB80233800EC
:100BE4001B016946009301F0C9FB320038000A2159
:100BF40001F024FC320038000B2101F01FFC80209E
:100C04003100C00301F01AFE286801F029FC0B49E9
:100C14000B4B28680B60CC604C608C600C614C61A1
:100C24008C6101F037FC3100286801F065FC28680C
:100C340001F06BFCAC80F7BD00040048B00200205A
:100C4400220C941070B5064C064D074B20002B6007
:100C540001F006FC2900200001F01CFC70BDC04618
:100C640000580040B00200202309720070B5064C01
:100C7400064D074B20002B6001F0F2FB29002000F9
:100C840001F008FC70BDC04600580040B0020020CE
:100C9400220C9410F8B506000F000C4D0C4B2B6081
:100CA4003900306801F051FC00280CD12C68631E17
:100CB4002B60002CF4D1B38830680133B38001F089
:100CC40024FC200000E00120F8BDC0460400002000
:100CD40010270000F0B587B00293838804000593C1
:100CE40080239B0100934E0031000068150000230F
:100CF400012201F013FC02212000FFF7CBFF0028A2
:100D040001D100209CE02900206801F019FC402159
:100D14002000FFF7BFFF0028F3D0FF210C98FFF756
:100D2400D9F9FF2107000C98FFF75AFA0D00002F9C
:100D340055D090239B01012F2BD1002929D1009359
:100D440080239B04FF223100206801F0E7FB029B13
:100D54000493FF330293039304212000FFF79AFFC7
:100D64000028CED0206801F0EDFB049B18700133FD
:100D74000493049A029B9342EED1013F002F0CD0BE
:100D840080212000FFF786FF0028BAD0012F53D01E
:100D94000023009380235B04D4E7002D3AD0802104
:100DA4002000FFF777FF0028ABD08023EAB29B0432
:100DB40000973100206801F0B1FB029B5D1904210A
:100DC4002000FFF767FF00289BD0206801F0BAFBE2
:100DD400039B187001330393AB42F0D11AE09023C4
:100DE4009B0100938023CAB29B043100206801F068
:100DF40095FB029E7519AE420CD004212000FFF72A
:100E040049FF002800D17CE7206801F09BFB30708B
:100E14000136F0E720212000FFF73CFF002800D135
:100E24006FE72068202101F097FB059BA088C01A7A
:100E340043425841C0B203E0002DA9D100957FE799
:100E440007B0F0BD70477047F0B5037985B007006F
:100E540002AC41791B4E022B0FD1012523000095D2
:100E6400FC223000FFF736FF092379796B440095A3
:100E7400FB223000FFF72EFF1DE0022303AD009399
:100E84001B222B003000FFF725FF2B7830001A01BE
:100E94006B781B11D3182370012379790B220093EB
:100EA4002B00FFF717FF04212B789A081140082222
:100EB4001A408B186370607823780002181880B287
:100EC40005B0F0BDCC020020F0B50500304C85B073
:100ED4002000FFF76BFE2000FFF7C8FE206801F03A
:100EE40014FB2B79022B2AD1052601273E336B7183
:100EF4006979009703ABFC222000FFF7EBFE002882
:100F040001D101203FE0013EF6B2002EF0D12000D5
:100F1400FFF798FE052601276979009703ABFC22A9
:100F24002000FFF7D7FE002803D12000FFF79EFE24
:100F340003E0013EF6B2002EEED1002023E036237A
:100F4400052601276B716979009703AB1B222000EA
:100F5400FFF7C0FE0028D4D0013EF6B2002EF2D135
:100F64002000FFF76FFE052601276979009703AB80
:100F74001B222000FFF7AEFE0028D6D0013EF6B2B9
:100F8400002EF2D1D9E70023A38005B0F0BDC046FE
:100F9400CC02002030B5037985B0417903AC1948FF
:100FA400194D022B10D10093FE222300FFF792FE6D
:100FB40000281FD058352B88207801339BB22B8012
:100FC4006378800118181BE002230C22009323008D
:100FD400FFF780FE00280DD058352B882078013388
:100FE4009BB22B80F02300021B0118406378181871
:100FF400800005E0002054352B8801339BB22B8000
:1010040005B030BDCC020020DC020020034B044AB2
:101014001A60044B044A083313607047CC02002062
:1010240000580040B4320008D40200207621C3697D
:1010340010B51A688A431A608022996952020A40DC
:101044001400611E8C41811CCC77002A07D17C21BD
:101054000132FF3242841A680A431A600AE0418C62
:10106400421DD1777A211A680A431A609A6979393C
:101074000A439A6101212E3002788A4302700822C1
:10108400DA6110BD1022C36970B5996911420DD19E
:101094009A69120702D5FFF7C9FF38E0202299693F
:1010A400114203D19A6992070ED430E0DA6159688B
:1010B400174A0A4076215A601A688A431A601A68E5
:1010C40012310A431A6022E001002E310A78D20755
:1010D4000CD4441DE27F856A561CE677FF243F2A20
:1010E40003D85200AA181488A4B284850A78D207B7
:1010F400D20FD2B280182C300278012004009A62F8
:101104000B78DA07D20F9443834323430B7070BDEB
:10111400FF7FFFFF1022C36970B599690400114273
:1011240001D0DA6159E09A69120702D5FFF77EFF10
:1011340053E09A69520704D42022996911422BD1B1
:101144004BE08022418C5200914204D15B6A63845B
:101154000534E37741E022002E32596A1378DB0725
:10116400DB0FDBB2E3182C3319701378DB0709D5D6
:10117400611DCB7FA06A5D1CCD771F2B02D8A18D8A
:101184005B001952012004001378D907C90F8C435E
:1011940083432343137020E0DA6103002E331B786A
:1011A400DB0712D5631DDB7FA16AFF223F2B03D827
:1011B4005A008A18128892B2200012122D3002703E
:1011C4001F2B02D8A28D5B005A52618C636BC9B28B
:1011D400A06A9847638F0133638770BDFA22C3699D
:1011E40010B59969114204D01968803A0A407A2AE4
:1011F4000BD0FC22996911420AD07C2219680A405A
:101204007C2A05D1FFF786FF0BE0FFF73BFF08E0E0
:1012140008229969114204D01B68134201D0FFF7D8
:1012240005FF10BD802310B5134C5B00E069826993
:101234001A4202D00268120610D48023E069DB004F
:1012440082691A4202D0026812060ED42000FFF707
:10125400C5FF0A4B228E56331A8010BDC361238EFC
:101264000133238601F051F9E7E7C361238E01338B
:10127400238601F04AF9E9E75C030020DC02002040
:101284001721064B064ADA615A1CD1778022520094
:101294005A84044A9A62044A5A6370475C030020E1
:1012A40000540040DC0200202513000810B5044B54
:1012B4000A000100186800F023F9002010BDC046A0
:1012C400A803002013B5144B041E1B68019310D00F
:1012D400012418001C70002100F05CF921000F4863
:1012E40001F052FC902022000421C00501F0A0F876
:1012F4000FE0020090200421C00501F099F82100BC
:10130400019800F047F9019B21001C70034801F08B
:101314003BFC002016BDC046A8030020002C014061
:1013240010B5030008292AD80800FEF7C9FE0505F0
:101334000C0E131F24281A005888198880B289B209
:10134400FFF7B4FF1CE09B8819E0D88880B2FFF750
:10135400B9FF15E019890B4B89B21868FEF756FFDF
:101364000DE0188A80B2FFF72FF908E0054B1868E2
:10137400FEF75EFF03E0034B1868FEF753FF0020FF
:1013840010BDC04644000020704700207047002074
:101394007047704780200649064A0B1D4002D867F3
:1013A4005832138801339BB21380086000207047C1
:1013B40000E100E0DC02002010B5040080200421DC
:1013C400C00501F0D9FC8020C00501F0D3FC80B237
:1013D400E080E3889BB2002B13D08020C00501F08D
:1013E400C7FC6423E188584389B2FEF773FE80B2D8
:1013F4002081E188044B89B21868FEF76BFEE06037
:1014040001E02381E36010BD1800002010B50248FC
:10141400FFF7D2FF10BDC04698030020024B034AD9
:10142400083313607047C046D04200089803002078
:10143400F0B50024047080202E4B2F4E8DB05C80BC
:1014440001211C80000101F0EDF9300001F0C4FA23
:10145400684601F077FB294B6A4601936B461C8072
:101464001C81202369463000538001F02FFB0423A4
:10147400012707ADAB8029005C3330002B806F80DF
:10148400AC81EC812C826C82099401F08BFB3000DE
:10149400082101F057FC2900300001F0C1FB3000A5
:1014A400082101F055FC2900300001F003FC300054
:1014B400082101F057FC802303AD1B012B808023FE
:1014C400DB006B8080235B00AB802900E93B3000AC
:1014D400EB802C81AC8101F047FB3900300001F036
:1014E4003AFB0D2328002B706F70AF7001F058F891
:1014F4000DB0F0BDDC020020002C01407604000099
:10150400037870B5002B33D01A48131C824201D9DA
:10151400194B1B88194A1A4C8A180C1992B2A4B296
:101524001848521164114911520064004900155AB7
:10153400095A245A9BB25D435C434B43124A124EF0
:10154400AD189B19114A2D0CA4191B0C5543534378
:10155400240C5443190C0E482D0C01F0EDFB240C03
:1015640029000B4801F0EAFB2100094801F0E8FBDF
:1015740070BDC04670FD0000EC42000855550000E7
:10158400AAAAFFFFD032000800008F0276040000F0
:10159400002C014070B50D00064C200001F0CCFB7E
:1015A4002900200001F0CAFB2900200001F0C8FB3B
:1015B40070BDC046002C0140014A024B1A607047BE
:1015C400AC030020A80300207047704710B5040046
:1015D40090201021C00500F029FF0220FEF77CFFB7
:1015E40021000C4801F09AF901210A4801F0B8F9E8
:1015F4000028F9D00820FEF76FFF90201021C005C5
:1016040000F012FF0520FEF767FF024801F08AF997
:1016140010BDC0460030014010B5040090201021D8
:10162400C00500F003FF0120FEF756FF21000C481F
:1016340001F076F901210A4801F092F90028F9D065
:101644000120FEF749FF90201021C00500F0ECFEB8
:101654000120FEF741FF024801F067F910BDC046C2
:101664000030014070B50124114E3470FFF7D4FFEF
:101674000020FFF7D1FF8023DB01034011D1850453
:10168400AD0C08D02B126B4019114B4099104B40F4
:1016940059104B402340C013434001200340337092
:1016A40003E00448FFF7B8FF0025280070BDC046DA
:1016B400C00300200140000070B50124104D2C70BF
:1016C400FFF7AAFF0223034013D1821091B2002A2C
:1016D40009D083125A4012B2131153409E10734022
:1016E4005A105340234001221040434013402B70B2
:1016F40004E0E7200002FFF78FFF0021080070BD1F
:10170400C0030020F0B5050087B000910D22002130
:1017140002A801F029FD02AB1D703E4B1B78002B83
:1017240003D002AB9E1C052401E0032402AE642D09
:1017340009D002D8002D08D068E02B00733B023496
:10174400012B01D962E00134E4B20021324801F0F6
:10175400D1F80021304801F0F5F801212E4801F0BC
:10176400F1F801212C4801F0C5F890200027102140
:10177400C00500F05BFE0220FEF7AEFE01970221D9
:10178400254801F0EDF80028F9D002ABF95C2248B5
:1017940001F0C4F80121204801F0E2F80028F9D052
:1017A4001D4801F0BFF802ABF854A31EBB4204D19C
:1017B400194B988AC043C3B201930137FBB29C42D0
:1017C400DDD890201021C00500F02EFE642D0DD030
:1017D40005D8002D1AD1337872781B0209E0733DC5
:1017E400012D13D8B378F2781B0202E03378023368
:1017F40000E0D318009A138002ABE418013C019B6B
:101804002078C01A43425841C0B200E0002007B01B
:10181400F0BDC046C103002000300140F7B5134CB1
:101824002378002B04D1C820FEF770FE0123237017
:1018340001260A250E4C26706B4600200D4F991D7B
:101844003870FFF75FFF002802D0002323700AE0FE
:101854006B46991D3E70FFF755FF0028F5D1013DF9
:10186400EDB2002DE8D12078FEBDC046C2030020B1
:10187400C0030020C1030020F0B50600802087B01B
:101884000121400100F0CEFFC0200121C00200F080
:10189400BDFF022301AC23710323002563710823D8
:1018A400202721005B480193A571E57100F066FDD6
:1018B40021005848019700F061FD102301930F3B6C
:1018C400A371022321005348E37100F057FD2A005D
:1018D4000321504800F0B2FD2A0004214D4800F0D5
:1018E400ADFD2A0005214B4800F0A8FD90201021F1
:1018F400C00500F099FD90203900C00500F094FD6A
:1019040090204021C00500F08FFD01239020237119
:1019140010232100C00501936571A571E57100F0E4
:101924002DFD90202100C005019700F027FD902097
:1019340040232100C005019300F020FD200000F0A9
:10194400A1FFE023DB00A3800123A7812381337956
:10195400012B03D01A00083A012A03D8F0231B01F3
:10196400A38002E0032B00D12581822300255B00A4
:101974006380FC3363816A3BFF3B2100264823825A
:10198400E5802580E58100F08BFF2900224800F0E6
:10199400CFFF80212048490100F0B6FF01211E48F5
:1019A40000F0A8FFFA204000FEF796FD02F0D0FCFC
:1019B4003379B060012B06D12800FFF72DFE1748BC
:1019C400FFF750FE21E0032B10D16424013C0020DA
:1019D400E4B2FFF7FBFD002C03D0A528F6D10020CC
:1019E40015E0A538431E9841C0B210E00A2B02D17D
:1019F400FFF714FF0BE0E7200002FFF70DFE084895
:101A0400FFF70AFE0548FFF757FE064B187807B0A4
:101A1400F0BDC0460004004800300140FFFF000054
:101A2400F0FF0000C003002037B56B4600259C1D65
:101A3400210028002580FFF765FE064BA84202D04E
:101A44002288920702D401221A7000E01D702088B7
:101A540080083EBDC0030020F8B5037906003B4D65
:101A6400012B03D13A48FFF7FDFD3AE0032B34D1B3
:101A7400023B00202B70FFF7A9FD060010281BD1A4
:101A84000020FFF7A3FD04003000FFF79FFDF023C3
:101A9400234005D1A40280002E4A204310802B70DD
:101AA4000020FFF793FD2C4BA5284AD01A78511C2F
:101AB4001970132AF4D944E0A5280BD1264A1378C7
:101AC400591C1170142B03D91020FFF77FFD01E07E
:101AD40000232B701F4B1C8822E00A2B03D1FFF735
:101AE400A3FF04001CE002F033FCB3681B4FC01AD0
:101AF400FA235B00984210D91548FFF7DDFD3379CE
:101B0400082B02D10001164C01E0164C8000044061
:101B140002F01EFC3C80B06002E000233C882B7085
:101B24002A78114B002A06D054331A880024013233
:101B340092B21A8008E058331A88013292B21A809D
:101B440002E000221A70C5E72000F8BDC00300209F
:101B5400FFFF0000AE030020B2030020B00300200A
:101B6400F03F0000FC3F0000DC0200200023F7B53A
:101B7400164F74203B706B469E1D3100FFF7C2FD6B
:101B8400002801D101233B700A213088FEF7A2FA14
:101B9400310085B26420FFF7B5FD002801D101238F
:101BA4003B703488310024070020A40FFFF7AAFDFE
:101BB400002801D101233B700C233088EDB2800052
:101BC4001840204300024019FEBDC046C003002057
:101BD400F8B500242B4E050034700379012B11D184
:101BE4002948FFF73FFD3378A3423FD1801184B2E7
:101BF4002648FFF737FD3378002B34D1FF33984361
:101C040024182FE0032B38D00A2B03D1FFF7AEFFA3
:101C1400040028E002F09CFBAB68C01AF423FF33F5
:101C24009842F7D91A48FFF7F7FC1A48FFF744FD22
:101C340033780700002B19D11748FFF73DFD33789F
:101C4400002B13D1C024BF00A400FF330440BB43C6
:101C5400E41880231B010340E21880238010DB007A
:101C640018401418A4B23378002B06D00B4A0A4C3F
:101C74005432138801339BB2138002F069FBA860CD
:101C84002000F8BDC0030020FE7F0000FD7F00009F
:101C9400F0FF0000B5E60000FFFF0000DC020020BA
:101CA400024B034A083313607047C046F0420008F1
:101CB400B403002010B5FEF70FFF10BD10B502F0FD
:101CC40047FB0F4A0F491368C31A8B4217D90E4BAF
:101CD40010605A8F0D4B1988914209D080219020B1
:101CE4000901C0051A8000F098FB0022012800D0E9
:101CF4000122802190200901C00500F099FB10BD4C
:101D0400C8030020400D03005C030020C40300202E
:101D1400704786239B00C35AC018007D704700009B
:101D24008622034B9200C35A805A181AC0B27047D5
:101D34001A0200008523044A9B00C35A825AFF20DA
:101D44009B1A98437047C0461602000087239B00E5
:101D5400C35CC018024BC018012303707047C0460F
:101D64001D02000010B5040023682000DB689847BA
:101D740000280AD0236820005B6898473E2804D0D6
:101D8400236820001B689847EEE7FEF723FB10BD8D
:101D940070B504000D00236820001B6998470028D3
:101DA400F9D085239B00E25AA218FF325575E268E8
:101DB400517D1F2211401E3A100088400A49C8670D
:101DC400E15A891889B2E152E15AC9B2E152074B8A
:101DD400186088239B00E35C002B03D104496068EE
:101DE40001F0A3F870BDC04604E100E000E100E0AA
:101DF40007010700862370B59B00C25A04008218AD
:101E0400157DC268517D1F2211401E3A8A400D493A
:101E1400CA670D4AC15A825A914207D0C25A013246
:101E240092B2C252C25AD2B2C25201E0FEF7D2FA00
:101E3400E36828005A7D1F231A401E3B9340034A3F
:101E4400136070BD04E100E01A02000000E100E04C
:101E540030B5037A87B0013BDBB20400042B03D80E
:101E6400214A9B009D5801E0E1256D020021606834
:101E740001F052F8606800F083FF00230293059399
:101E840023690095049387239B00E35CDBB2002B5A
:101E940005D080235B0101938023DB0000E00193E4
:101EA40069466068039300F0DBFF802160684901A4
:101EB40001F054F885220D4B9200E35A60689BB2FE
:101EC400A35286239B00E35A094A9BB2A3520022E1
:101ED400084B01211A7101F01FF8012206496068BC
:101EE40001F023F807B030BD3043000816020000AB
:101EF4001A020000A00200200501050030B504000C
:101F0400236187232272002208009B00E160E254CF
:101F140085B00A7D0069097B00F090FA022302ADC6
:101F24002B7101336B71E36829005A891869029295
:101F34000122AA71EA7100F021FAE36858680028C6
:101F440001D10422226122690C2A0DD11A7A9978CE
:101F540000F074FAE36829001A8858680292002293
:101F6400AA71EA7100F00AFAE36801A85B7D0370C4
:101F740003234370023B837000F012FB2000FFF741
:101F840067FF05B030BD000010B5064800F0E6FA62
:101F9400032000F0E9FA012000F0ECFA00F0F0FA76
:101FA40010BDC0465555000010B500F0F1FA10BD43
:101FB400F7B5102000F05AFB80200121C00200F088
:101FC40025FC8020012180030124022700F036FC37
:101FD40003256B461F715D719C71DC71402369465A
:101FE4004F48009300F0CAF9802369464C48009397
:101FF40000F0C4F922000621494800F01FFA22002B
:102004000721474800F01AFA80202100800200F0DE
:1020140015FC80202100800200F0F8FBC020210084
:10202400C00200F0F3FB6B4600265D7190251F7122
:102034009E71DC718023ED0528005B0069460093E6
:1020440000F09CF9802328006946009300F096F97B
:10205400802328009B006946009300F08FF96946AD
:102064002F48009400F08AF980232800DB00694699
:10207400009300F083F969462948009700F07EF93F
:102084003A002800082100F0D9F93A002800072175
:1020940000F0D4F93A002800092100F0CFF93A0001
:1020A40031001F4800F0CAF93A0028000A2100F064
:1020B400C5F93A0021001A4800F0C0F96B465E7178
:1020C4009E711C71042328006946009300F056F9A0
:1020D40080202100800200F099FB6B461E715E7126
:1020E4009E71DF71202328006946009300F046F9B1
:1020F400402328006946009300F040F98020210025
:10210400800200F083FB6B465E719E71DE711C7170
:10211400802328001B016946009300F02FF9F7BDC6
:1021240000040048024A1388013313807047C046F4
:102134007C02002070B59025ED052800402100F0B8
:1021440065F920210400280000F060F964002043B0
:10215400C0B270BD7FB58D21394B00259A1CD18743
:102164001A0079394E3211805D811D8154331D80EE
:10217400FEF7EEF9FFF71CFFFEF79CF9FFF704FFEB
:10218400FEF764F9FFF7D6FF2E4C06002300E06942
:1021940038331D7000F064F9802319361B02636123
:1021A400F6B2294B2100E06976002360E5606560A2
:1021B400A5602661A56100F06DF90121E06900F0D8
:1021C4009BF9631CDB7F03A80370012345708370B4
:1021D40000F0E6F9E3691D4A596825860A4076212C
:1021E4005A601A688A431A601A6812310A431A60DC
:1021F400174B1B6818000193FEF700F8154B18687D
:10220400FFF716F96420FEF781F902F0A1F8040043
:102214000198FEF753F8104B0A211888421C1A80C3
:10222400FDF7DEFF0D4B89B219700D4B8900CB58B9
:10223400984702F08DF8001B6328FAD9E5E7C046F9
:10224400DC0200205C030020220C9410FF7FFFFFBF
:1022540044000020A80300207E0200208002002009
:10226400703200087047FEE770477047074B70B53F
:1022740000251E00064CE41AA410A54204D0AB00AD
:10228400F35898470135F8E770BDC046B8440008D4
:10229400D8440008074B10B5984209D18020012189
:1022A400800000F0D7FA80200021800000F0D2FAEC
:1022B40010BDC0460024014030B58A680D68C3686B
:1022C4001543CA68064C15430A69234015434A69F5
:1022D40015432A001A430B795B031343C36030BDD3
:1022E40003D2FFFF0023036003718360C3600361B3
:1022F4004361704783680122002900D102221343FD
:1023040083607047836A1943816242617047802108
:10231400826809060A43F0210300826009029A6870
:102324000139D20FD207002901D0002AF7D10020A9
:102334009A68824200DB186C704704228368134356
:1023440083607047006C80B270474368002A02D0F3
:102354001943416001E08B4343607047CB0103D5CF
:102364008068044B184000E000680840411E884122
:10237400C0B27047FFFFFFFE01607047F7B50B68FE
:102384000193002301249C40019A224094422CD1C1
:102394000A79551E012D15D85E00B44603266746FA
:1023A400BE408568B54385604E798568BE402E433E
:1023B40086608588A54385808C7985889C402C43DC
:1023C400A4B2848003245D00AC40E443AA400668C0
:1023D40026400660066832430260C2681440C46046
:1023E400CA79C468AA402243C2600133102BC9D100
:1023F400F7BD0000044B0122036000234271037106
:102404008371C3717047C046FFFF0000038A1940FF
:102414000800411E8841C0B27047838A19400800F1
:10242400411E8841C0B27047816170470185704781
:10243400002A01D0816100E001857047072310B5AF
:102444000F240B409B009C409A40C9088900401807
:10245400016AA1430162016A0A43026210BD0000DD
:102464000B4B10B50121984207D18020800300F066
:10247400FDF980200021800306E08020C00300F0E5
:10248400F5F980200021C00300F0F0F910BDC0462A
:102494000054004030B5012403688A68A3430360F4
:1024A40003681502114A13404A682B43134303601F
:1024B4000F4A0B681A40026103680A6923430360E8
:1024C40000238360C3608B69134380228360836825
:1024D4001202134383600368CA68134303604268AB
:1024E400044B13404A691343436030BDFFE0CF00FF
:1024F400FFFFFFF0FF7FFF0701220368002901D0DF
:10250400134300E0934303607047012102688A4348
:102514000260036803680B430360704730B514001E
:102524004568064A89052A40039D890D2A431343B9
:102534000B4322041A43426030BDC046009800FC9D
:1025440081627047406AC0B27047836919400800CD
:10255400411E8841C0B27047C1617047014B186089
:102564007047C04600300040014B58607047C04679
:1025740000300040014B98607047C0460030004076
:10258400014A024B1A607047AAAA000000300040BA
:10259400014A024B1A607047CCCC00000030004066
:1025A400837870B50178002B1BD08B08104A032662
:1025B4009B009B18FF223140B1401600C0248E407E
:1025C400A4001D59B5434678B60132408A402A43D7
:1025D4001A511F2302781A401E3B9340044A136089
:1025E40005E01F2319401E3B8B40024AD36770BD90
:1025F40000E100E004E100E00121114B1A680A4304
:102604001A6058680F4A02405A6018680E4A02401D
:102614001A6018680D4A02401A6058680C4A024051
:102624000F205A60DA6A8243DA62186B094A024060
:102634001A635A6B8A435A6300229A607047C046F1
:10264400001002400CB8FFF8FFFFF6FEFFFFFBFF8F
:10265400FFFFC0FFACFEF0FF0321034A53688B4326
:10266400184350607047C046001002401021044BCC
:102674001A6B8A431A631A6B104318637047C04677
:1026840000100240F8B50C23594D04006868184046
:10269400FDF716FD1F1F1F1F1F1F1F1F071F1F1FD3
:1026A4001D000F21C02368686A68800C08405B0223
:1026B400861C1A4201D14F4806E04D4B4E48DB6A56
:1026C40019400131FDF706FD7043206004E04B4BD7
:1026D40000E0494B0020236021686B680A00484EE3
:1026E4001B061B0FF35CDA40130062606A68520534
:1026F400520FB25CD340A3602A6BD20501D4414A85
:1027040006E03B4A5268520401D45A0800E09A0891
:10271400E2602A6B520601D43B4A01E08022120295
:1027240022612A6BD20602D4334A626100E06161FD
:1027340003222F6B2E4E174201D1A36112E0376B97
:102744001740012F01D1A1610CE0376B1740022F14
:1027540002D18022120204E0366B3240032A01D1F6
:10276400254AA261C0222F6B9202174201D1E36174
:1027740019E01F4E376B802617407602B74201D10D
:10278400E16110E01A4E376B80261740B602B7425B
:1027940002D18022120205E0154E366B1640964295
:1027A40001D1154AE261C0222F6B1203104E174269
:1027B40015D08027336BFF021340BB4201D1216245
:1027C4000EE08021336B090313408B4202D1802336
:1027D4001B0204E0336B1340934201D1064B236286
:1027E4002B6B1B0602D4054B636200E06062F8BDEC
:1027F4000010024000093D0000127A00006CDC0267
:1028040008000020809FD50012800000044B5A6904
:10281400002902D01043586101E082435A61704795
:1028240000100240044B9A69002902D010439861B9
:1028340001E082439A61704700100240044BDA6958
:10284400002902D01043D86101E08243DA61704765
:1028540000100240044BDA68002902D01043D8600B
:1028640001E08243DA60704700100240044B1A69A9
:10287400002902D01043186101E082431A617047B5
:10288400001002400023E02203804380D200C38072
:10289400038143818381C38107338280038270472C
:1028A400C12310B504889B010A881C40CB891343BB
:1028B400CA8813430A8913434A8913438A891343F1
:1028C400234303808288094B13408A8813430422DC
:1028D40083800B8A0382038893434A8813430380CB
:1028E400828B034B1340838310BDC046FFF0FFFF70
:1028F400FFF7FFFF40220388002901D0134300E0C3
:1029040093430380704700008288034B1340838005
:102914008388194381807047FFEFFFFF017370477D
:1029240081817047007BC0B27047808980B2704754
:102934000288034B134003800388194301807047C6
:10294400FFF7FFFF002904D080220388920113437C
:1029540002E00288014B134003807047FFDFFFFF52
:10296400038919400800411E8841C0B27047000025
:10297400054B1A68042802D11043186002E00421B0
:102984008A431A607047C04610E000E0014B58606B
:102994007047C04610E000E0084B012803D11A68D4
:1029A4001043186008E0821C04D101211A688A438C
:1029B4001A6001E000229A607047C04610E000E00F
:1029C400044B02211A68002801D00A4300E08A431C
:1029D4001A60704710E000E0344B10B5984208D1FB
:1029E400802001210001FFF735FF80200021000134
:1029F40059E08023DB05984206D101210800FFF746
:102A040035FF0021012028E0294B984206D10121FD
:102A14000220FFF72BFF002102201EE0254B9842E5
:102A240006D101211020FFF721FF0021102014E01E
:102A3400214B984206D101212020FFF717FF0021E6
:102A440020200AE01D4B98420AD180200121400039
:102A5400FFF70CFF802000214000FFF707FF24E070
:102A6400174B984208D1802001214002FFF7F2FE63
:102A740080200021400216E0124B984208D18020A9
:102A840001218002FFF7E6FE8020002180020AE097
:102A94000D4B984209D180200121C002FFF7DAFED4
:102AA40080200021C002FFF7D5FE10BD002C01409C
:102AB40000040040001000400014004000200040CA
:102AC40000400140004401400048014030B5038803
:102AD400154C9BB2A04206D08022D205904202D06F
:102AE400124A904203D1702293434A881343104AF6
:102AF400904203D00F4A0D8913402B4303804B6847
:102B0400C3620B880385A04208D00B4B984205D0C2
:102B14000A4B984202D00A4B984201D18B7A038621
:102B24000123838230BDC046002C014000040040D4
:102B340000100040FFFCFFFF004001400044014042
:102B44000048014001235B4243600023038003816A
:102B540043808372704701220388002901D0134304
:102B640000E09343038070470A884B880630134380
:102B74008A881343CA8813430A8913434A8913432F
:102B84008A891343C38770470630002904D0802301
:102B9400C28F1B02134302E0C38F5B045B0CC38729
:102BA40070470000012270B57324038C934303849F
:102BB400038C8288058B92B2A5430C88254302249A
:102BC400A3431E004C888B892343104C3343A042FB
:102BD40008D00F4CA04205D00E4CA04202D00E4C9F
:102BE400A0420DD10824A343CC890E8A2343042494
:102BF400A3438C882343094C22404C8A3443224308
:102C040082808A6805834263038470BD002C01407E
:102C1400004001400044014000480140FFFCFFFF28
:102C24001022038C70B593430384048C1C4A83885C
:102C3400058B0E881540202294438A89360212019E
:102C440014434A8835431201A4B2164E14439BB26E
:102C5400ADB2A2B2B04202D0134CA04219D1134C6F
:102C640023400C8AA40023439BB2B04211D1802498
:102C7400A243CC89240114434022A4B294438A88F9
:102C840012011443A2B20A4C23404C8AA4002343E9
:102C94009BB283808B6805838363028470BDC046C6
:102CA400FF8CFFFF002C014000400140FFFBFFFFB1
:102CB400FFF7FFFF028C1A4B70B513400384732394
:102CC400048C8288858B8E899D430B8836021D4334
:102CD400144B92B21C404B8834431B02A4B21C43D5
:102CE400A3B2114CA04214D1104C2340CC8924022D
:102CF40023430F4C23408C88240223430D4C9BB266
:102D040022400C8A2401224394B24A8A12011443B9
:102D1400A2B282808A688583C263038470BDC04680
:102D2400FFFEFFFFFFFDFFFF002C0140FFF7FFFF49
:102D3400FFFB0000FFCFFFFF4163704781637047D3
:102D4400C16370470822038B93431943018370477F
:102D5400028B034B09021340194389B20183704764
:102D6400FFF7FFFF0822838B934319438183704746
:102D7400406B7047806B7047C94389B201827047CA
:102D84002F4B10B5984208D180200121C001FFF7D4
:102D940061FD80200021C0014EE02A4B984208D1F9
:102DA400802001218002FFF761FD80200021800244
:102DB40022E0254B984208D180200121C002FFF770
:102DC40055FD80200021C00216E0204B984208D116
:102DD400802001210003FFF749FD8020002100032A
:102DE4000AE01B4B98420AD1802001214003FFF7DF
:102DF4003DFD802000214003FFF738FD1EE0154B08
:102E0400984206D101212020FFF724FD0021202033
:102E140012E0114B984206D101214020FFF71AFD20
:102E24000021402008E00D4B984207D10121802069
:102E3400FFF710FD00218020FFF70CFD10BDC046F8
:102E4400003801400044004000480040004C00406D
:102E5400005000400014014000180140001C0140D3
:102E64000122F0B50D0003688BB093430360426800
:102E7400224B040013408A68134343600268204BCA
:102E84001A404B68C9680B4329690B431343036019
:102E940082681C4B13406A69134383606846FFF7DA
:102EA400F1FB194B069E9C4208D0184B079E9C428E
:102EB40004D0174B089E9C4200D0029E23682F68C2
:102EC4001B0400D5760039003000FDF703F9390002
:102ED40005003000FDF784F900237F08B9425B4107
:102EE400ED1823681B0404D50A4B2A07520F1D4012
:102EF4001543ADB2A5810BB0F0BDC046FFCFFFFFB7
:102F0400F3E9FFFFFFFCFFFF0038014000440040ED
:102F140000480040F0FF000001220368002901D0AE
:102F2400134300E0934303607047FF2310B50C1272
:102F34001C401940FE3B8B40022C01D1043002E0BE
:102F4400032C00D10830002A02D00268134302E0A7
:102F540002689A431300036010BD00008268034BAB
:102F6400134083608368194381607047FFEFFFFF5C
:102F7400FF230A121A400B4010B51C000123A34082
:102F8400012A01D1026804E0022A01D1426800E06A
:102F940082681340C2690020834206D0090C0130C4
:102FA40088401040431E9841C0B210BD1348854666
:102FB40004200168090E1F22914205D11048012105
:102FC4000160104800210160002103E00E4B5B58B2
:102FD400435004310D480E4B42189A42F6D30D4A21
:102FE40002E00023136004320B4B9A42F9D300F041
:102FF40017F8FFF73BF9FFF7ADF8FEE700200020D4
:103004001810024000000140D844000800000020CD
:103014001C0000201C000020CC030020FEE7000060
:1030240013B50121474B1A680A431A605868464A87
:1030340002405A601868454A02401A601868444AB7
:1030440002401A605868434A02400F205A60DA6A04
:103054008243DA62186B404A02401A635A6B80203A
:103064008A435A63002280219A60009201921A686E
:1030740049020A43A0211A608002C9011A68024069
:103084000192009A01320092019A002A02D1009A18
:103094008A42F3D18022186892022A49024002D05F
:1030A4000122019204E0019208682C4A02400A605D
:1030B40011202B49019C086059682A4A59605968B3
:1030C400596059680A405A605A68012C1CD18821F9
:1030D40049030A4380215A601A6849040A4380213B
:1030E4001A6089041868174A0842FBD00320516803
:1030F4008143516051680138014351600C215A6881
:103104000A40082AFBD11BE0A02189030A4380213D
:103114005A601A6849040A4380211A6089041868AD
:10312400084A0842FBD0032051688143516051682A
:103134000138014351600C215A680A40082AFBD126
:1031440013BDC046001002400CB8FFF8FFFFF6FEA6
:10315400FFFFFBFFFFFFC0FFACFEFFFFFFFFFEFF13
:1031640000200240FF7FC0FF70B583073FD0541E8C
:10317400002A3BD0CEB20300032503E0621E002CDC
:1031840034D0140001335A1E16702B42F6D1032C8E
:1031940024D9FF250D402A0215432A0415430F2C78
:1031A40011D92600103E3609013636011A009B1942
:1031B400156055609560D56010329342F8D10F22A6
:1031C4001440032C0AD9261FB6080136B6001A008B
:1031D4009B1920C29342FCD103221440002C05D039
:1031E400C9B21C19197001339C42FBD170BD140083
:1031F4000300CCE70000000000000000F10100081B
:10320400F5010008F7010008FB010008FD010008B2
:1032140020000020B4030020D4020020B4030020C6
:10322400980300209803002084020020D402002088
:10323400B4030020B4030020B40300200000000005
:1032440000000000F5030008030400081D04000842
:103254003304000800400E00000000480100008014
:103264000F00000000000048011C0000B91C000809
:10327400C11C0008151D00084B0500084D05000879
:103284004F050008510500085305000849050008CA
:10329400292100080000000000000000E5050008E6
:1032A4008D060008C1060008E3050008DF050008D4
:1032B4000000000000000000CD0E00084B0E0008C6
:1032C400990F0008490E00084D0E0008FF7F648026
:1032D400C8802D819181F6815A82BF82238388839D
:1032E400EC835184B5841A857E85E2854786AB8656
:1032F40010877487D8873D88A18805896989CE8914
:10330400328A968AFA8A5E8BC38B278C8B8CEF8CDD
:10331400538DB78D1B8E7F8EE28E468FAA8F0E90B3
:103324007190D59039919C9100926392C7922A939F
:103334008E93F1935494B8941B957E95E19544969D
:10334400A7960A976D97CF9732989598F8985A99B7
:10335400BD991F9A819AE49A469BA89B0A9C6C9CEF
:10336400CE9C309D929DF49D569EB79E199F7A9F48
:10337400DC9F3DA09EA0FFA060A1C1A122A283A2C8
:10338400E4A245A3A5A306A466A4C7A427A587A56C
:10339400E7A547A6A7A607A766A7C6A725A885A841
:1033A400E4A843A9A2A901AA60AABFAA1EAB7CAB48
:1033B400DBAB39AC98ACF6AC54ADB2AD10AE6DAE7F
:1033C400CBAE29AF86AFE3AF40B09DB0FAB057B1F2
:1033D400B4B110B26DB2C9B225B382B3DEB339B49D
:1033E40095B4F1B44CB5A7B503B65EB6B9B614B787
:1033F4006EB7C9B723B87DB8D8B832B98BB9E5B9B7
:103404003FBA98BAF1BA4BBBA4BBFDBB55BCAEBC2A
:1034140006BD5FBDB7BD0FBE67BEBEBE16BF6DBFE6
:10342400C4BF1CC072C0C9C020C176C1CDC123C2F3
:1034340079C2CFC224C37AC3CFC324C479C4CEC44F
:1034440023C577C5CCC520C674C6C8C61BC76FC7FD
:10345400C2C715C868C8BBC80EC960C9B3C905CA04
:1034640057CAA8CAFACA4BCB9CCBEDCB3ECC8FCC67
:10347400DFCC30CD80CDD0CD1FCE6FCEBECE0DCF24
:103484005CCFABCFFACF48D096D0E4D032D180D144
:10349400CDD11AD267D2B4D201D34DD39AD3E6D3C5
:1034A40031D47DD4C8D414D55FD5A9D5F4D53ED6AE
:1034B40089D6D2D61CD766D7AFD7F8D741D88AD801
:1034C400D2D81BD963D9ABD9F2D93ADA81DAC8DABE
:1034D4000EDB55DB9BDBE1DB27DC6DDCB2DCF8DCEF
:1034E4003DDD81DDC6DD0ADE4EDE92DED6DE19DF8D
:1034F4005CDF9FDFE2DF24E067E0A9E0EAE02CE1A3
:103504006DE1AEE1EFE130E270E2B0E2F0E230E32F
:103514006FE3AEE3EDE32CE46BE4A9E4E7E424E534
:1035240062E59FE5DCE519E655E692E6CEE609E7B5
:1035340045E780E7BBE7F6E731E86BE8A5E8DFE8B5
:1035440018E951E98AE9C3E9FCE934EA6CEAA3EA37
:10355400DBEA12EB49EB80EBB6EBECEB22EC58EC3C
:103564008DECC2ECF7EC2CED60ED94EDC8EDFCEDC8
:103574002FEE62EE95EEC7EEFAEE2BEF5DEF8FEFD6
:10358400C0EFF1EF21F052F082F0B1F0E1F010F170
:103594003FF16EF19CF1CAF1F8F126F253F280F298
:1035A400ADF2DAF206F332F35DF389F3B4F3DFF349
:1035B40009F434F45EF487F4B1F4DAF403F52CF589
:1035C40054F57CF5A4F5CBF5F2F519F640F666F65C
:1035D4008CF6B2F6D7F6FDF621F746F76AF78EF7C2
:1035E400B2F7D6F7F9F71CF83EF861F883F8A4F8B7
:1035F400C6F8E7F808F928F949F969F988F9A8F942
:10360400C7F9E5F904FA22FA40FA5EFA7BFA98FA65
:10361400B5FAD1FAEDFA09FB25FB40FB5BFB76FB1F
:1036240090FBAAFBC4FBDDFBF7FB0FFC28FC40FC72
:1036340058FC70FC87FC9EFCB5FCCCFCE2FCF8FC5E
:103644000DFD23FD38FD4CFD61FD75FD88FD9CFDE0
:10365400AFFDC2FDD4FDE7FDF9FD0AFE1CFE2DFE03
:103664003DFE4EFE5EFE6EFE7DFE8CFE9BFEAAFEC1
:10367400B8FEC6FED4FEE1FEEEFEFBFE08FF14FF1C
:1036840020FF2BFF36FF41FF4CFF56FF60FF6AFF10
:1036940073FF7CFF85FF8EFF96FF9EFFA5FFACFFA7
:1036A400B3FFBAFFC0FFC6FFCCFFD1FFD7FFDBFFDC
:1036B400E0FFE4FFE8FFEBFFEFFFF2FFF4FFF6FFAC
:1036C400F8FFFAFFFCFFFDFFFDFFFEFFFEFFFEFF1C
:1036D400FDFFFDFFFCFFFAFFF8FFF6FFF4FFF2FF2A
:1036E400EFFFEBFFE8FFE4FFE0FFDBFFD7FFD1FFD5
:1036F400CCFFC6FFC0FFBAFFB3FFACFFA5FF9EFF20
:1037040096FF8EFF85FF7CFF73FF6AFF60FF56FF05
:103714004CFF41FF36FF2BFF20FF14FF08FFFBFE89
:10372400EEFEE1FED4FEC6FEB8FEAAFE9BFE8CFEB3
:103734007DFE6EFE5EFE4EFE3DFE2DFE1CFE0AFE6E
:10374400F9FDE7FDD4FDC2FDAFFD9CFD88FD75FDCF
:1037540061FD4CFD38FD23FD0DFDF8FCE2FCCCFCC5
:10376400B5FC9EFC87FC70FC58FC40FC28FC0FFC5C
:10377400F7FBDDFBC4FBAAFB90FB76FB5BFB40FB8A
:1037840025FB09FBEDFAD1FAB5FA98FA7BFA5EFA51
:1037940040FA22FA04FAE5F9C7F9A8F988F969F9AF
:1037A40049F928F908F9E7F8C6F8A4F883F861F8A4
:1037B4003EF81CF8F9F7D6F7B2F78EF76AF746F732
:1037C40021F7FDF6D7F6B2F68CF666F640F619F652
:1037D400F2F5CBF5A4F57CF554F52CF503F5DAF404
:1037E400B1F487F45EF434F409F4DFF3B4F389F349
:1037F4005DF332F306F3DAF2ADF280F253F226F21D
:10380400F8F1CAF19CF16EF13FF110F1E1F0B1F081
:1038140082F052F021F0F1EFC0EF8FEF5DEF2BEF6C
:10382400FAEEC7EE95EE62EE2FEEFCEDC8ED94EDE8
:1038340060ED2CEDF7ECC2EC8DEC58EC22ECECEBEB
:10384400B6EB80EB49EB12EBDBEAA3EA6CEA34EA71
:10385400FCE9C3E98AE951E918E9DFE8A5E86BE87E
:1038640031E8F6E7BBE780E745E709E7CEE692E60D
:1038740055E619E6DCE59FE562E524E5E7E4A9E41D
:103884006BE42CE4EDE3AEE36FE330E3F0E2B0E2AB
:1038940070E230E2EFE1AEE16DE12CE1EAE0A9E0B3
:1038A40067E024E0E2DF9FDF5CDF19DFD6DE92DE33
:1038B4004EDE0ADEC6DD81DD3DDDF8DCB2DC6DDC2A
:1038C40027DCE1DB9BDB55DB0EDBC8DA81DA3ADA95
:1038D400F2D9ABD963D91BD9D2D88AD841D8F8D771
:1038E400AFD766D71CD7D2D689D63ED6F4D5A9D5BC
:1038F4005FD514D5C8D47DD431D4E6D39AD34DD36F
:1039040001D3B4D267D21AD2CDD180D132D1E4D08E
:1039140096D048D0FACFABCF5CCF0DCFBECE6FCE12
:103924001FCED0CD80CD30CDDFCC8FCC3ECCEDCBF7
:103934009CCB4BCBFACAA8CA57CA05CAB3C960C93B
:103944000EC9BBC868C815C8C2C76FC71BC7C8C6DD
:1039540074C620C6CCC577C523C5CEC479C424C4D7
:10396400CFC37AC324C3CFC279C223C2CDC176C127
:1039740020C1C9C072C01CC0C4BF6DBF16BFBEBECB
:1039840067BE0FBEB7BD5FBD06BDAEBC55BCFDBBBB
:10399400A4BB4BBBF1BA98BA3FBAE5B98BB932B9FB
:1039A400D8B87DB823B8C9B76EB714B7B9B65EB680
:1039B40003B6A7B54CB5F1B495B439B4DEB382B34C
:1039C40025B3C9B26DB210B2B4B157B1FAB09DB05B
:1039D40040B0E3AF86AF29AFCBAE6DAE10AEB2ADA3
:1039E40054ADF6AC98AC39ACDBAB7CAB1EABBFAA28
:1039F40060AA01AAA2A943A9E4A885A825A8C6A7E4
:103A040066A707A7A7A647A6E7A587A527A5C7A4CE
:103A140066A406A4A5A345A3E4A283A222A2C1A1ED
:103A240060A1FFA09EA03DA0DC9F7A9F199FB79E36
:103A3400569EF49D929D309DCE9C6C9C0A9CA89BA6
:103A4400469BE49A819A1F9ABD995A99F898959839
:103A54003298CF976D970A97A7964496E1957E95ED
:103A64001B95B8945494F1938E932A93C7926392BE
:103A740000929C913991D59071900E90AA8F468FA7
:103A8400E28E7F8E1B8EB78D538DEF8C8B8C278CA3
:103A9400C38B5E8BFA8A968A328ACE8969890589B4
:103AA400A1883D88D88774871087AB864786E285CE
:103AB4007E851A85B5845184EC8388832383BF82F1
:103AC4005A82F68191812D81C8806480FF7F9A7F1C
:103AD400367FD17E6D7E087EA47D3F7DDB7C767C47
:103AE400127CAD7B497BE47A807A1C7AB77953796E
:103AF400EE788A782678C1775D77F9769576307690
:103B0400CC7568750475A0743B74D77373730F73A5
:103B1400AB724772E3717F711C71B8705470F06FAF
:103B24008D6F296FC56E626EFE6D9B6D376DD46CA3
:103B3400706C0D6CAA6B466BE36A806A1D6ABA6985
:103B44005769F46891682F68CC6769670667A4664B
:103B54004166DF657D651A65B8645664F4639263F3
:103B64003063CE626C620A62A8614761E56084607A
:103B74002260C15F605FFF5E9E5E3D5EDC5D7B5DDB
:103B84001A5DB95C595CF85B985B375BD75A775A16
:103B9400175AB7595759F75898583858D957795721
:103BA4001A57BB565C56FD559E553F55E0548254FA
:103BB4002354C55366530853AA524C52EE519151A3
:103BC4003351D55078501B50BE4F614F044FA74E10
:103BD4004A4EEE4D914D354DD94C7C4C204CC54B45
:103BE400694B0D4BB24A574AFB49A0494549EA483B
:103BF40090483548DB4781472647CC4673461946EB
:103C0400BF4566450D45B3445A440144A943504356
:103C1400F8429F424742EF4197414041E84091407A
:103C24003A40E23F8C3F353FDE3E883E313EDB3D4D
:103C3400853D2F3DDA3C843C2F3CDA3B853B303BD1
:103C4400DB3A873A323ADE398A393639E3388F3803
:103C54003C38E93796374337F0369E364B36F935DC
:103C6400A73556350435B33462341134C0336F3359
:103C74001F33CE327E322E32DF318F314031F1307C
:103C8400A23053300430B62F682F1A2FCC2E7E2E3C
:103C9400312EE42D972D4A2DFD2CB12C642C182C9B
:103CA400CD2B812B362BEA2A9F2A552A0A2AC02992
:103CB40075292C29E22898284F280628BD2774271F
:103CC4002C27E3269B2653260C26C4257D25362542
:103CD400F024A92463241D24D72391234C230623F1
:103CE400C1227D223822F421B0216C212821E52033
:103CF400A2205F201C20DA1F971F551F141FD21EFD
:103D0400911E501E0F1ECE1D8E1D4E1D0E1DCE1C4F
:103D14008F1C501C111CD21B931B551B171BDA1A2A
:103D24009C1A5F1A221AE519A9196C193019F51889
:103D3400B9187E1843180818CD17931759171F1769
:103D4400E616AD1674163B160216CA1592155B15C7
:103D54002315EC14B5147E1448141214DC13A613A2
:103D640071133C130713D2129E126A1236120212F6
:103D7400CF119C11691137110411D310A1106F10C8
:103D84003E100D10DD0FAC0F7C0F4D0F1D0FEE0E0E
:103D9400BF0E900E620E340E060ED80DAB0D7E0DC6
:103DA400510D240DF80CCC0CA10C750C4A0C1F0CF5
:103DB400F50BCA0BA00B770B4D0B240BFB0AD20A95
:103DC400AA0A820A5A0A330A0C0AE509BE099809A2
:103DD40072094C0927090109DD08B808940870081C
:103DE4004C0828080508E207C0079D077B075A0707
:103DF40038071707F606D606B5069506760656065C
:103E040037061906FA05DC05BE05A0058305660517
:103E140049052D051105F504D904BE04A30488043D
:103E24006E0454043A0421040704EF03D603BE03CA
:103E3400A6038E0377036003490332031C030603BE
:103E4400F102DB02C602B2029D028902760262021C
:103E54004F023C022A0217020502F401E201D101D9
:103E6400C101B001A00190018101720163015401FB
:103E7400460138012A011D0110010301F600EA0080
:103E8400DE00D300C800BD00B200A8009E0094006C
:103E94008B008200790070006800600059005200B5
:103EA4004B0044003E00380032002D002700230060
:103EB4001E001A00160013000F000C000A00080070
:103EC40006000400020001000100000000000000E0
:103ED4000100010002000400060008000A000C00B2
:103EE4000F00130016001A001E00230027002D00E7
:103EF400320038003E0044004B005200590060007C
:103F040068007000790082008B0094009E00A80075
:103F1400B200BD00C800D300DE00EA00F6000301D1
:103F240010011D012A013801460154016301720187
:103F340081019001A001B001C101D101E201F401AC
:103F4400050217022A023C024F026202760289022B
:103F54009D02B202C602DB02F10206031C03320315
:103F64004903600377038E03A603BE03D603EF035E
:103F7400070421043A0454046E048804A304BE0410
:103F8400D904F50411052D05490566058305A00529
:103F9400BE05DC05FA0519063706560676069506AB
:103FA400B506D606F606170738075A077B079D0796
:103FB400C007E207050828084C0870089408B808E8
:103FC400DD08010927094C0972099809BE09E509A8
:103FD4000C0A330A5A0A820AAA0AD20AFB0A240BD6
:103FE4004D0B770BA00BCA0BF50B1F0C4A0C750C71
:103FF400A10CCC0CF80C240D510D7E0DAB0DD80D7D
:10400400060E340E620E900EBF0EEE0E1D0F4D0FF7
:104014007C0FAC0FDD0F0D103E106F10A110D310EC
:104024000411371169119C11CF11021236126A1250
:104034009E12D21207133C137113A613DC1312142D
:1040440048147E14B514EC1423155B159215CA1587
:1040540002163B167416AD16E6161F17591793175A
:10406400CD17081843187E18B918F51830196C19AB
:10407400A919E519221A5F1A9C1ADA1A171B551B7B
:10408400931BD21B111C501C8F1CCE1C0E1D4E1DCD
:104094008E1DCE1D0F1E501E911ED21E141F551FA5
:1040A400971FDA1F1C205F20A220E52028216C2105
:1040B400B021F42138227D22C12206234C239123EE
:1040C400D7231D246324A924F02436257D25C42563
:1040D4000C2653269B26E3262C277427BD27062867
:1040E4004F289828E2282C297529C0290A2A552AFC
:1040F4009F2AEA2A362B812BCD2B182C642CB12C29
:10410400FD2C4A2D972DE42D312E7E2ECC2E1A2FE8
:10411400682FB62F04305330A230F13040318F3144
:10412400DF312E327E32CE321F336F33C03311343F
:104134006234B33404355635A735F9354B369E36DB
:10414400F03643379637E9373C388F38E338363919
:104154008A39DE39323A873ADB3A303B853BDA3BFF
:104164002F3C843CDA3C2F3D853DDB3D313E883E8F
:10417400DE3E353F8C3FE23F3A409140E8404041CB
:104184009741EF4147429F42F8425043A9430144BB
:104194005A44B3440D456645BF4519467346CC465B
:1041A40026478147DB4735489048EA484549A049B6
:1041B400FB49574AB24A0D4B694BC54B204C7C4CCA
:1041C400D94C354D914DEE4D4A4EA74E044F614F9B
:1041D400BE4F1B507850D55033519151EE514C5233
:1041E400AA5208536653C55323548254E0543F558E
:1041F4009E55FD555C56BB561A577957D9573858B2
:104204009858F7585759B759175A775AD75A375BA6
:10421400985BF85B595CB95C1A5D7B5DDC5D3D5E67
:104224009E5EFF5E605FC15F22608460E5604761FF
:10423400A8610A626C62CE6230639263F46356646E
:10424400B8641A657D65DF654166A46606676967BB
:10425400CC672F689168F4685769BA691D6A806AE7
:10426400E36A466BAA6B0D6C706CD46C376D9B6DF6
:10427400FE6D626EC56E296F8D6FF06F5470B870ED
:104284001C717F71E3714772AB720F737373D773D1
:104294003B74A07404756875CC7530769576F976A0
:1042A4005D77C17726788A78EE785379B7791C7A66
:1042B400807AE47A497BAD7B127C767CDB7C3F7D23
:1042C400A47D087E6D7ED17E367F9A7F000000003B
:1042D40000000000931300089713000899130008C6
:1042E4008D1300088F13000870FD0000000000000B
:1042F400000000007D180008CF1500085D1A0008B2
:10430400CD150008D51B00080000000000000000C7
:10431400F91D0008171D0008951D0008251D00083B
:10432400391D0008691D0008511D000800E1000046
:1043340000960000004B00008025000000E8030008
:1043440010B5024800F048F810BDC0464C000020EB
:104354000A4A0B4970B595680C689268094B08685D
:10436400954203D95C430621280003E04343062118
:104374001C001000FBF7AEFE201A70BD10E000E038
:104384000000002040420F00044A13680133136008
:10439400034A1368013313607047C04600000020CD
:1043A4007802002010B50948FDF7CCFF084B0949F5
:1043B4009A898A4204D001329A819A6810189860C6
:1043C40004210248FDF7D8FF10BDC0460024014077
:1043D40084020020FFFF000070B52F4904004068EC
:1043E400FEF7C6FD00282FD063682C489D8CDA693F
:1043F400ADB292070DD18621294A8900835A415AC8
:104404000133DBB28B421BD0815A835241180D75A4
:104414001AE0DA6987239B00D20702D4C25C002A1F
:104424000ED18722C35C1F49C3185B181B78920006
:10443400002B05D10121835C4B408354FDF708FD1B
:10444400194A13880133138018496068FEF790FDF8
:1044540000281FD08522114B9200985A144A995A69
:1044640088420CD0995A60685918FF31497D0185FA
:10447400995A013189B29952995AC9B299528521EE
:1044840089009A5A5B5A9A4204D10022074960680B
:10449400FEF74BFD70BDC046050105004C00002031
:1044A4001A0200001D020000480000200701070056
:0444B40016020000EC
:1044B800B9030008A1040008150700081110000836
:1044C8008512000821140008BD150008A51C000865
:1044D8000100000010270000000000000102030492
:0C44E8000102030406070809006CDC0256
:0400000508002FB10F
:00000001FF
